:100000002AEF0FF020202020202020202020202058
:100010002020202000002D2D2D2D2D2D2D2D2D2D9E
:100020002D2D000025372E34664D204F686D0000C1
:1000300025372E33666B204F686D000025382E3231
:1000400066204F686D002D2D2D2D2D005220202073
:100050000000453234200000202020200000EA6A01
:10006000480EE96EEF500DE00A0E016E006A002E98
:10007000FED7012EFBD75F0E006E002EFED7EF2EAF
:10008000F3D7120093909392939493969398939AA4
:1000900089969296929E898A929A8B8094808B8878
:1000A00094888B8A948A8B8C948C8B8E948E8B8282
:1000B00094828B8494848B869486C050C00B0709ED
:1000C000C06EC08EC2800F015C51800B5C6F010E50
:1000D0005D6FC196C198C19A000E016EC250830B2C
:1000E0000110C26E000E016EC150F80B0110C16EFE
:1000F000870ECD6EAA6A00014EEF0FF0899A5A6AF8
:100100005A500F0812E3000B006E5950800B036E1B
:100110000050031002E0898E01D0899E898689965D
:10012000D890583659365A2AEBD7898ACAEF00F048
:100130005450010A0FE0030A0FE0060A10E0010A1A
:1001400011E00D0A12E0020A13E01A0A14E0300A64
:1001500015E018D0556A16D0010E556E13D0020E58
:10016000556E10D0030E556E0DD0040E556E0AD08C
:10017000050E556E07D0060E556E04D0070E556E4F
:1001800001D0556A55C056F0400E576E596E55C095
:1001900058F0B4D7120062A902D08A8001D08A90A8
:1001A00062A702D08A8A01D08A9A62A502D08A8880
:1001B00001D08A9862A302D08A8601D08A9662A171
:1001C00002D08A8401D08A9412008A8200D08A9256
:1001D00000D01200640E486E42DF030E626FDBDF58
:1001E000F4DF050E486E3BDF030E626FD4DFEDDFF8
:1001F000010E486E34DF030E626FCDDFE6DF010EC5
:10020000486E2DDF020E626FC6DFDFDF010E486E23
:1002100026DF020E626FBFDFD8DF010E486E1FDFE0
:100220000E0E626FB8DFD1DF010E486E18DF626B11
:10023000B2DFCBDF010E486E12DF080E626FABDF5C
:10024000C4DF010E486E0BDF626BA5DFBEDF010E5F
:10025000486E05DF0C0E626F9EDFB7DF010E486E41
:10026000FEDE626B98DFB1DF010E486EF8DE060E2F
:10027000626F91DFAADF010E486EF1DE626B8BDFE9
:10028000A4DF010E486EEBDE010E626F84DF9DDF9E
:10029000020E486EE4DE58EF0FF0626B7CDF95DFF4
:1002A000020E626F78DF91DF020E486ED8DE5AEFE1
:1002B0000FF05450000A07E0010A0EE0030A15E0AF
:1002C000010A1CE024D094909498949A949C949E53
:1002D0009482948494861BD0949294809488948A77
:1002E000948C948E9484948612D094949480948860
:1002F000948A948C948E9482948609D09496948057
:100300009488948A948C948E9482948400D0120061
:10031000C2825B90C2A25B805BB004D05B90C2A241
:100320005B80FAD7C2B2FED7C4CF03F0C3CF5CF074
:10033000C4CF5DF05CC001F05DC002F0A9EF01F038
:10034000576A566A556A546A586A58503F080CE30F
:10035000DFD702C003F00150542602505522000E90
:1003600056225722582AF1D7573256325532543234
:100370005732563255325432573256325532543241
:100380005732563255325432573256325532543231
:100390005732563255325432030E571655C05AF062
:1003A00054C059F059C001F05AC002F01200526A0C
:1003B000010E536E52500508D8A0AED052500BE03B
:1003C000010A0DE0030A0FE0010A11E0070A13E039
:1003D000010A15E018D0010E546EAADE14D0020EE8
:1003E000546EA6DE10D0040E546EA2DE0CD0080EA1
:1003F000546E9EDE08D0100E546E9ADE04D0200E8D
:10040000546E96DE00D0010E536E546A52DF1A0EFF
:10041000006E002EFED7000093DF02C04BF001C03B
:100420004AF0010E546E45DF1A0E006E002EFED704
:10043000000086DF02C04DF001C04CF0020E546E89
:1004400038DF1A0E006E002EFED7000079DF02C0E2
:100450004FF001C04EF0030E546E2BDF1A0E006EEB
:10046000002EFED700006CDF02C051F001C050F03A
:100470005250080DF350556A546E040E5424E96E20
:10048000000E5520EA6E4BC0ECFFED524AC0EFFF64
:100490005250080DF350556A546E020E5424016EEA
:1004A000000E5520036E0150040FE96E000E03206C
:1004B000EA6E4DC0ECFFED524CC0EFFF5250080DFC
:1004C000F350556A546E040E5424016E000E5520EC
:1004D000036E0150040FE96E000E0320EA6E4FC058
:1004E000ECFFED524EC0EFFF5250080DF350556A2D
:1004F000546E060E5424016E000E5520036E0150FA
:10050000040FE96E000E0320EA6E51C0ECFFED52BD
:1005100050C0EFFF522A4ED75CEF0FF0100E516E15
:10052000506A4A6A4A50050857E34B6A4B50030821
:1005300051E34A50080DF350536A526ED8904B3431
:10054000036A5224016E535003220150040FE96ED6
:10055000000E0320EA6EECCF4DF0ED52EFCF4CF0E1
:100560004D5003080AE2FF0A03E14C50000805E27F
:10057000000E4C5E040E4D5A05D0000ED8804C562D
:10058000040E4D564D50515C23E303E150504C5C3A
:100590001FE24AC048F04BC049F04DC051F04CC07A
:1005A00050F04A50080DF350536A526ED8904B34B5
:1005B000036A5224016E535003220150040FE96E66
:1005C000000E0320EA6EECCF39F0ED52EFCF38F099
:1005D0004B2AACD74A2AA6D748C036F049C037F0D4
:1005E0005EEF0FF08E0E006E55C001F054C002F0A9
:1005F000036A015209E102C001F0026A080E005EBE
:10060000015202E1006A08D0D89001BE04D002363F
:1006100001360006F9D7019EDAEF05F06451D8B42F
:1006200071D0006E6851D8B46DD0002604E3810EFD
:10063000002668E204D07F0E005E64E363E065C0DC
:100640006CF069516C1B658F698F67516B03F4CF38
:100650006EF066516A03F4CF03F0F3CF6DF06B03D5
:10066000F3506E27F4506D23000E032267516A0386
:10067000F3506E27F4506D23000E026A032202220B
:1006800065516B03F3506D27F4500322000E0222D4
:1006900065516A03F3500326F4500222000E016AEA
:1006A000012267516903F3506D27F4500322000EB5
:1006B0000222012266516903F3500326F4500222FC
:1006C000000E012265516903F3500226F450012205
:1006D000002A01BE05D06D3703360236013600060A
:1006E000000E6DAF0AD0032A02220122015005E15B
:1006F000025003E1035001E1002A6CBF018E6CAF90
:10070000019E04D0006A016A026A036A1200800E28
:10071000D8B2611B666B676B5DC065F06151651B8C
:100720005C50D8B4DCD0646F006E6051D8B4E0D0B7
:10073000645FD8B481D03DE361C06AF06A8F62C063
:1007400069F063C068F0676BD8906A3369336833C7
:100750006733642FF8D765AF03D06681DDD066912B
:1007600064916689EA6A5F0EE96EE9D0669965BFB1
:100770000AD064A113D06A33693368336733002A1F
:10078000D8B4C5D00BD06ABF0CD0D89067376837C3
:1007900069376A370006D8B4BAD0F5D7668D6BD002
:1007A000669D5DC065F05DAE02D06A8FA9D06A9F7C
:1007B000A7D060C064F060C000F05C50645F5DC0B2
:1007C0006AF06A8F5EC069F05FC068F0676BD890AE
:1007D0006A33693368336733642FF8D765AF03D062
:1007E00066839AD066936491668BEA6A630EE96EBB
:1007F000A6D0669B65BF0AD064A113D06A33693363
:1008000068336733002AD8B482D00BD06ABF0CD0CB
:10081000D8906737683769376A370006D8B477D019
:10082000F5D7668F28D0669F61C065F061AF02D0B2
:100830006A8F66D06A9F64D061C06AF06A8F62C0B6
:1008400069F063C068F065AF04D06A9F668564D0C4
:100850006695676B6491EA6A5F0EE96E70D065BF5A
:100860001CD05DC065F064A106D06A33693368337B
:100870006733002A4CE067AF0BD0682B09E1692B86
:1008800007E16A2B05E16A3369336833002A3FE0E8
:1008900066BD86D766BFC7D71CD0800E6A1B6AAFFD
:1008A00004D03AD061C065F00AD05DC065F06A53EB
:1008B00006E1695304E1685302E1006A21D06ABF8E
:1008C00008D0D8906737683769376A37002EF7D76E
:1008D0001ED065AF02D06A8F13D06A9F11D060C05E
:1008E00000F061C06AF062C069F063C068F008D0CF
:1008F0005CC000F05DC06AF05EC069F05FC068F087
:100900006AC001F069C002F068C003F034D0006A28
:10091000016A026A036A2FD0676B681F691F6A1F2A
:10092000671F672B05E1682B03E1692B01E16A2B47
:1009300066B115D766B356D766B58AD7B3D7EF5029
:10094000682705E3692B03E16A2BD8B46481ED5273
:10095000EF50692703E36A2BD8B46481ED52EF505E
:10096000EFBE01D0800A6A27D8B0648166B9FED68E
:1009700066BB3FD774D723EF06F05850D8B4A5D044
:10098000646F5C50D8B4A1D0645F05E37F0E642728
:10099000D8B09BD006D0810E645FD8A096D0D8B4D2
:1009A00094D064C000F0016A026A036A636B59C0A4
:1009B00062F0628F5AC061F05BC060F0190E646F24
:1009C0005F50605F0DE2010E615F0AE2625F08E264
:1009D000635F06E2632B622B612B5F50602728D098
:1009E0005E50615F12E2010E625F0FE2635F0DE233
:1009F000632B622B5E5061275F50602719E3612BE8
:100A000017E1622B15E1632B13D05D508009625F03
:100A10000EE2010E635F0BE2632B5D5080096227DB
:100A20005E506127E9E3622BE7E1632BE5D70380A2
:100A3000642F01D00BD0D8906037613762376337AD
:100A4000D8900336023601366537BAD765A106D08D
:100A5000D890013202320332653302D0000635E00D
:100A600065BF1ED0D89060376137623763375F50FB
:100A7000605F07E2010E615F04E2625F02E2635FB2
:100A80001AE35E50615F05E2010E625F02E2635F9E
:100A900012E35D508009625F03E2010E635F0BE3C6
:100AA000032A09E1022A07E1012A05E1002A0DE0F3
:100AB00001320232033259C064F05D50641B64AFEE
:100AC00002D0018E06D0019E04D0006A016A026A3B
:100AD000036A12003750000A07E0010A0CE0030A1B
:100AE00012E0010A18E01FD04B6A4A6A7A0E496E7A
:100AF000890E486E18D04B6A400E4A6E1C0E496E25
:100B00008C0E486E10D04B6A500E4A6E430E496EE2
:100B10008F0E486E08D04B6A240E4A6E740E496ED2
:100B2000920E486E00D036500BE0010A0FE0030A27
:100B300013E0010A17E0070A1BE0010A1FE024D0B6
:100B40004F6A4E6A4D6A7F0E4C6E1ED04F6A4E6AD7
:100B50004D6A800E4C6E18D04F6A4E6A4D6A810EF7
:100B60004C6E12D04F6A4E6A4D6A820E4C6E0CD09B
:100B70004F6A4E6A4D6A830E4C6E06D04F6A4E6ABB
:100B80004D6A840E4C6E00D039500D080EE2FF0AFB
:100B900003E138508B0809E2800E536E960E526EB8
:100BA000180E516E960E506E67D039C055F038C091
:100BB00054F018D503C053F002C052F001C051F0F8
:100BC00000C050F053C067F052C066F051C065F0ED
:100BD00050C064F04BC06BF04AC06AF049C069F085
:100BE00048C068F01BDD03C057F002C056F001C0DA
:100BF00055F000C054F0676B666B656B8B0E646FCD
:100C00004FC06BF04EC06AF04DC069F04CC068F048
:100C100005DD03C05BF002C05AF001C059F000C00E
:100C200058F0D88203C05FF002C05EF001C05DF0F2
:100C300000C05CF053C063F052C062F051C061F07C
:100C400050C060F064D557C05BF056C05AF055C034
:100C500059F054C058F003C05FF002C05EF001C00C
:100C60005DF000C05CF089DE03C053F002C052F0BA
:100C700001C051F000C050F050C000F051C001F070
:100C800052C002F053C003F060EF0FF04C38006E1A
:100C90000F0E001600500F0B4E6E4C500F0B4D6E8A
:100CA0004EC062F0CBEC00F0E5EC00F06A0E006E96
:100CB000002EFED700004DC062F0CBEC00F0E5EC5A
:100CC00000F06A0E006E002EFED7000081EF06F0E5
:100CD0004950000A07E0010A06E0030A07E0010A9A
:100CE00008E00AD009D0400E482606D0140E482647
:100CF00003D0540E482600D0800E48244B6E4C6E14
:100D0000C5D712005F38606F0F0E60175F16100EA8
:100D10006025616F626FCBEC00F0E5EC00F0100E27
:100D20005F24616F626FCBEC00F0E5EC00F06A0EBF
:100D3000006E002EFED7000012000900F5520CE0F4
:100D4000F6CF52F0F7CF53F0F5CF5FF0DBDF52C0B4
:100D5000F6FF53C0F7FFF1D7120053C05AF05750B7
:100D60005A1A5AAE05D0D894D89053BED8802FD0F6
:100D700053C05AF056C05BF052505B5E06E05AAE6C
:100D800026D0D850010AD86E22D057C05BF05350FD
:100D90005B5E06E05AAE1BD0D850010AD86E17D061
:100DA00058C05BF054505B5E06E05AAE10D0D8508D
:100DB000010AD86E0CD059C05BF055505B5E06E05E
:100DC0005AAE05D0D850010AD86E01D0D890120082
:100DD0005F50B6085F6E036A60C063F0608FD890A2
:100DE00060336133623303320232013200325F2EEC
:100DF000F6D763AF0BD0001E011E021E031E002A91
:100E0000D8B4012AD8B4022AD8B4032A77EF07F05D
:100E1000D8B203D0EA6A670EE96E006A016A026A14
:100E2000036A676B686B696B6A6B66516511641165
:100E300063112CE0200E6B6FD8905F3660376137FE
:100E400062376737683769376A3766516A5D08E124
:100E50006551695D05E16451685D02E16351675D5B
:100E60000FE36351675F6451D8A0643D685F6551CB
:100E7000D8A0653D695F6651D8A0663D6A5FD8809D
:100E800000360136023603366B2FD6D767C0EFFF28
:100E900068C0ECFF69C0ECFF6AC0ECFF1200E950CB
:100EA000576E5650596E1AE055C067F054C066F040
:100EB00053C065F052C064F06B6B6A6B200E696FB3
:100EC000820E686F0EEC03F003C055F002C054F0C0
:100ED00001C053F000C052F0592EE6D755C062F061
:100EE00054C061F053C060F052C05FF071D703C0CE
:100EF00055F002C054F001C053F000C052F055AE9E
:100F00000DD05706578A521E531E541E551E522A84
:100F1000D8B4532AD8B4542AD8B4552A3B0E5E6E9E
:100F20009A0E5D6ECA0E5C6E5B6A0A0E596E565062
:100F3000D8B4572AD882EA6A520EE96E55C062F0D8
:100F400054C061F053C060F052C05FF05EC066F004
:100F50005DC065F05CC064F05BC063F059DF0150B8
:100F600000520FE15628595C0CE057500CE00F0B73
:100F7000595C01E037E257BE35D057BC04D0200E93
:100F80002DD0200E571657AA0CD0579A5650D8A4D9
:100F900057060050576E2D0E5F6EB4DE5750006E30
:100FA000576A5650595C0AE10050576E2E0E5F6E1C
:100FB000A9DE5750006E200E5716000E300E57AAAD
:100FC0000DD0579A5650D8A457060050576E2D0E84
:100FD0005F6E98DE5750006E576A300E002600C0D4
:100FE0005FF090DED8925EC062F05DC061F05CC0E0
:100FF00060F05BC05FF0666B656B646B0A0E636FDD
:1010000007DF03C05EF002C05DF001C05CF000C00D
:101010005BF0592E8FD712000900F6CF51F0F7CFB1
:1010200052F0F5CF5FF06EDE51C0F6FF52C0F7FF11
:10103000502EF2D71200600E556EF50E546E100E43
:10104000536E960E526E4BC059F04AC058F049C0CC
:1010500057F048C056F081DE06E3160EF66E000E1D
:10106000F76E6BDE8FD0556AEF0E546E670E536EBF
:10107000920E526E4BC059F04AC058F049C057F01A
:1010800048C056F06ADE2DE34BC05BF04AC05AF010
:1010900049C059F048C058F05F6A240E5E6E740E65
:1010A0005D6E920E5C6E69DC03C04FF002C04EF0C4
:1010B00001C04DF000C04CF0060EE96E03C055F0C3
:1010C00002C054F001C053F000C052F0040E566E3E
:1010D000E6DE290EF66E000EF76E050E506E9CDFF2
:1010E00051D0556A700E546E140E536E8C0E526EA3
:1010F0004BC059F04AC058F049C057F048C056F0AC
:101100002CDE2CE34BC05BF04AC05AF049C059F0CA
:1011100048C058F05F6A5E6A7A0E5D6E880E5C6E3B
:101120002CDC03C04FF002C04EF001C04DF000C0F7
:101130004CF0060EE96E03C055F002C054F001C039
:1011400053F000C052F0030E566EA9DE350EF66E57
:10115000000EF76E050E506E5FDF14D0070EE96EBD
:101160004BC055F04AC054F049C053F048C052F04B
:10117000020E566E94DE410EF66E000EF76E040EF1
:10118000506E4ADF7CEF0FF08E0E006E6451005EF1
:1011900065C002F066C001F0028E005209E0D890EE
:1011A000025202E1015204E002320132002EF7D76E
:1011B00065AF05D0011E021E012AD8B4022A120012
:1011C00059C067F058C066F057C065F056C064F06B
:1011D0006B6B800E6A6F3B0E696F8A0E686F0EEC48
:1011E00003F003C061F002C060F001C05FF000C016
:1011F0005EF061C067F060C066F05FC065F05EC021
:1012000064F0C2DF02C063F001C062F063510B08FA
:101210000DE303E162512A0809E3C30E616FF50E85
:10122000606F680E5F6E7E0E5E6E2ED263510A088E
:1012300012E2FF0A03E162512A080DE263510C0831
:101240000AE303E162514E0806E3616B606B5F6A7B
:101250007F0E5E6E19D263510B0815E2FF0A03E19F
:1012600062514D0810E263510D080DE303E1625134
:101270007A0809E3CD0E616FCC0E606F0C0E5F6EC5
:101280007F0E5E6E01D263510C0815E2FF0A03E186
:101290006251790810E263510E080DE303E16251D7
:1012A000A60809E39A0E616F990E606F190E5F6EC2
:1012B0007F0E5E6EE9D163510D0814E2FF0A03E16F
:1012C0006251A5080FE2635110080CE303E162517B
:1012D000680808E3660E616F606F260E5F6E7F0E12
:1012E0005E6ED2D163510F0813E2FF0A03E162512F
:1012F00067080EE2635112080BE303E162512A080A
:1013000007E3616B606B400E5F6E7F0E5E6EBCD15B
:101310006351110815E2FF0A03E16251290810E246
:10132000635113080DE303E16251EC0809E3CD0EAC
:10133000616FCC0E606F4C0E5F6E7F0E5E6EA4D13F
:101340006351120813E2FF0A03E16251EB080EE257
:10135000635116080BE303E16251440807E3660E8C
:10136000616F606F5F6E7F0E5E6E8ED16351150888
:1013700012E2FF0A03E1625143080DE263511808CB
:101380000AE303E162519C0806E3616B606B5F6AEC
:10139000800E5E6E79D16351170815E2FF0A03E1F2
:1013A00062519B0810E263511A080DE303E1625198
:1013B000F40809E3CD0E616FCC0E606F0C0E5F6E0A
:1013C000800E5E6E61D16351190815E2FF0A03E1D8
:1013D0006251F30810E263511D080DE303E162510D
:1013E000E20809E39A0E616F990E606F190E5F6E45
:1013F000800E5E6E49D163511C0815E2FF0A03E1BD
:101400006251E10810E2635121080DE303E16251EA
:10141000660809E3CD0E616FCC0E606F2C0E5F6E17
:10142000800E5E6E31D16351200813E2FF0A03E1A2
:10143000625165080EE2635124080BE303E1625137
:10144000EA0807E3616B606B400E5F6E800E5E6EB4
:101450001BD16351230814E2FF0A03E16251E9083A
:101460000FE2635128080CE303E162516E0808E3C0
:10147000330E616F606F530E5F6E800E5E6E04D12F
:101480006351270813E2FF0A03E162516D080EE27F
:1014900063512B080BE303E16251F20807E3660E88
:1014A000616F606F5F6E800E5E6EEED063512A08D2
:1014B00015E2FF0A03E16251F10810E263513008BE
:1014C0000DE303E162510C0809E39A0E616F990E76
:1014D000606F790E5F6E800E5E6ED6D063512F08FE
:1014E00015E2FF0A03E162510B0810E26351340870
:1014F0000DE303E16251BC0809E39A0E616F990E96
:10150000606F090E5F6E810E5E6EBED06351330850
:1015100014E2FF0A03E16251BB080FE2635139088C
:101520000CE303E162516C0808E3660E616F606FC3
:10153000160E5F6E810E5E6EA7D06351380814E2FE
:10154000FF0A03E162516B080FE263513E080CE3AE
:1015500003E16251B20808E3330E616F606F230E3E
:101560005F6E810E5E6E90D063513D0813E2FF0AFC
:1015700003E16251B1080EE2635145080BE303E158
:101580006251240807E3330E616F606F5F6E810E56
:101590005E6E7AD06351440814E2FF0A03E162519F
:1015A00023080FE263514C080CE303E162512C085D
:1015B00008E3660E616F606F460E5F6E810E5E6EB1
:1015C00063D063514B0815E2FF0A03E162512B0817
:1015D00010E2635153080DE303E16251CA0809E3C5
:1015E0009A0E616F990E606F590E5F6E810E5E6E7E
:1015F0004BD06351520813E2FF0A03E16251C9085C
:101600000EE263515B080BE303E16251FE0807E35E
:10161000616B606B700E5F6E810E5E6E35D06351D4
:101620005A0814E2FF0A03E16251FD080FE2635118
:1016300065080CE303E162515E0808E3330E616F55
:10164000606F030E5F6E820E5E6E1ED06351640883
:1016500015E2FF0A03E162515D0810E263516F0871
:101660000DE303E16251EA0809E39A0E616F990EF6
:10167000606F110E5F6E820E5E6E06D0616B606BE6
:10168000200E5F6E820E5E6E5EC000F05FC001F0E5
:1016900060C002F061C003F01200EACF5AF0E9CF57
:1016A00059F053AE08D0598E59A8592A521E531ECC
:1016B000522AD8B4532A5338F009556E5526E20FF2
:1016C000566E320F586E53500F0B5626562658261C
:1016D000E90F576E5726572652380F0B57265826B4
:1016E00057365836581E583652500F0B5826553616
:1016F000070E546E0A0E57065826FDE35606572667
:10170000FDE355065626FDE354065526FDE3EA6A39
:10171000540EE96E070E5914599CED52591407E105
:1017200059B8EE5259B803D0200E006E20D0E926E9
:10173000000EEA22E950580803E1EA5201E1598C0F
:10174000EF50006E08E159BC06D059B81CD059B60C
:1017500002D0200E0BD059AE06D02D0E006EED50EB
:10176000599C599E04D059865998300E0026EACFCC
:1017700053F0E9CF52F000C05FF082EC06F053C0A6
:10178000EAFF52C0E9FFEE5059ACD4D712004BC06B
:1017900055F04AC054F049C053F048C052F0596A5D
:1017A000586A200E576E820E566EADEC06F062E35C
:1017B0004BC059F04AC058F049C057F048C056F0E5
:1017C000FFDC03C04FF002C04EF001C04DF000C07E
:1017D0004CF04FC055F04EC054F04DC053F04CC0CB
:1017E00052F0596A586A576A7F0E566EADEC06F091
:1017F00013E3030EE96E4FC055F04EC054F04DC0D8
:1018000053F04CC052F0020E566E4FEC07F0200E13
:101810005F6E82EC06F02DD04FC055F04EC054F0F4
:101820004DC053F04CC052F0596A586A200E576EA2
:10183000820E566EADEC06F00FE3030EE96E4FC05C
:1018400055F04EC054F04DC053F04CC052F0010E54
:10185000566E4FEC07F00DD0030EE96E4FC055F0F9
:101860004EC054F04DC053F04CC052F0566A4FEC8D
:1018700007F0EED24BC055F04AC054F049C053F0C7
:1018800048C052F0596A586A480E576E850E566E17
:10189000ADEC06F06AE34BC05BF04AC05AF049C0B9
:1018A00059F048C058F05F6A5E6A200E5D6E820E85
:1018B0005C6EBDEC04F003C055F002C054F001C0F2
:1018C00053F000C052F003C059F002C058F001C0FC
:1018D00057F000C056F074DC03C04FF002C04EF069
:1018E00001C04DF000C04CF04FC067F04EC066F034
:1018F0004DC065F04CC064F06B6B6A6B200E696F75
:10190000820E686F0EEC03F003C067F002C066F051
:1019100001C065F000C064F037DC02C051F001C0C6
:1019200050F04FC055F04EC054F04DC053F04CC075
:1019300052F0596A586A576A7F0E566EADEC06F03F
:101940000CE3020EE96E51C053F050C052F0A5DE18
:10195000200E5F6E82EC06F007D0020EE96E51C0D9
:1019600053F050C052F099DE73D24BC055F04AC0CC
:1019700054F049C053F048C052F0596A586A7A0E80
:10198000576E880E566EADEC06F070E34BC05BF000
:101990004AC05AF049C059F048C058F05F6A5E6AC0
:1019A000480E5D6E850E5C6EBDEC04F003C055F014
:1019B00002C054F001C053F000C052F003C059F00F
:1019C00002C058F001C057F000C056F0E0EC08F03B
:1019D00003C04FF002C04EF001C04DF000C04CF00B
:1019E0004FC067F04EC066F04DC065F04CC064F06B
:1019F0006B6B6A6B480E696F850E686F0EEC03F0B7
:101A000003C067F002C066F001C065F000C064F07A
:101A1000C4EC08F002C051F001C050F04FC055F0C6
:101A20004EC054F04DC053F04CC052F0596A586A41
:101A3000576A7F0E566EADEC06F00CE3020EE96EAF
:101A400051C053F050C052F028DE200E5F6E82EC81
:101A500006F00BD0020EE96E51C053F050C052F0A8
:101A60001CDE200E5F6E82EC06F0F2D14BC055F00A
:101A70004AC054F049C053F048C052F0596A400E71
:101A8000586E1C0E576E8C0E566EADEC06F060E371
:101A90004BC05BF04AC05AF049C059F048C058F0FA
:101AA0005F6A5E6A7A0E5D6E880E5C6EBDEC04F055
:101AB00003C055F002C054F001C053F000C052F012
:101AC00003C059F002C058F001C057F000C056F0F2
:101AD000E0EC08F003C04FF002C04EF001C04DF042
:101AE00000C04CF04FC055F04EC054F04DC053F004
:101AF0004CC052F0596A586A576A7F0E566EADEC68
:101B000006F013E3030EE96E4FC055F04EC054F0DB
:101B10004DC053F04CC052F0020E566E4FEC07F021
:101B20006B0E5F6E82EC06F012D0030EE96E4FC0B2
:101B300055F04EC054F04DC053F04CC052F0010E61
:101B4000566E4FEC07F06B0E5F6E82EC06F080D1A4
:101B50004BC055F04AC054F049C053F048C052F051
:101B6000596A500E586E430E576E8F0E566EADEC7E
:101B700006F071E34BC05BF04AC05AF049C059F01F
:101B800048C058F05F6A400E5E6E1C0E5D6E8C0E93
:101B90005C6EBDEC04F003C055F002C054F001C00F
:101BA00053F000C052F003C059F002C058F001C019
:101BB00057F000C056F0E0EC08F003C04FF002C050
:101BC0004EF001C04DF000C04CF04FC067F04EC069
:101BD00066F04DC065F04CC064F06B6B6A6B200E14
:101BE000696F820E686F0EEC03F003C067F002C0ED
:101BF00066F001C065F000C064F0C4EC08F002C0FB
:101C000051F001C050F04FC055F04EC054F04DC0DF
:101C100053F04CC052F0596A586A576A7F0E566E9C
:101C2000ADEC06F00CE3020EE96E51C053F050C06B
:101C300052F033DD6B0E5F6E82EC06F00BD0020EBD
:101C4000E96E51C053F050C052F027DD6B0E5F6E4D
:101C500082EC06F0FDD04BC055F04AC054F049C0AC
:101C600053F048C052F0596A240E586E740E576EE5
:101C7000920E566EADEC06F071E34BC05BF04AC0BD
:101C80005AF049C059F048C058F05F6A500E5E6E75
:101C9000430E5D6E8F0E5C6EBDEC04F003C055F01C
:101CA00002C054F001C053F000C052F003C059F01C
:101CB00002C058F001C057F000C056F0E0EC08F048
:101CC00003C04FF002C04EF001C04DF000C04CF018
:101CD0004FC067F04EC066F04DC065F04CC064F078
:101CE0006B6B6A6B480E696F850E686F0EEC03F0C4
:101CF00003C067F002C066F001C065F000C064F088
:101D0000C4EC08F002C051F001C050F04FC055F0D3
:101D10004EC054F04DC053F04CC052F0596A586A4E
:101D2000576A7F0E566EADEC06F00CE3020EE96EBC
:101D300051C053F050C052F0B0DC6B0E5F6E82ECBD
:101D400006F00BD0020EE96E51C053F050C052F0B5
:101D5000A4DC6B0E5F6E82EC06F07AD04BC055F0BF
:101D60004AC054F049C053F048C052F0800E596E3A
:101D7000960E586E180E576E960E566EADEC06F017
:101D800061E34BC05BF04AC05AF049C059F048C00B
:101D900058F05F6A240E5E6E740E5D6E920E5C6E7D
:101DA000BDEC04F003C055F002C054F001C053F084
:101DB00000C052F003C059F002C058F001C057F003
:101DC00000C056F0E0EC08F003C04FF002C04EF047
:101DD00001C04DF000C04CF04FC055F04EC054F063
:101DE0004DC053F04CC052F0596A586A576A7F0E82
:101DF000566EADEC06F013E3030EE96E4FC055F0DE
:101E00004EC054F04DC053F04CC052F0020E566E0E
:101E10004FEC07F04D0E5F6E82EC06F012D0030E11
:101E2000E96E4FC055F04EC054F04DC053F04CC059
:101E300052F0010E566E4FEC07F04D0E5F6E82ECC5
:101E400006F006D0460EF66E000EF76E9DEC06F01C
:101E500090EF0FF0F86AD09E600ED36E400E9B6E2E
:101E6000646A356A346A0F015C51800B5C6F000E46
:101E70005D6FC196C198C19A5E6B5F6B600ED36E49
:101E8000400E9B6E646AFF0E926E936E946E640EAB
:101E9000486E00012FEC00F042EF00F0640E486E37
:101EA0002FEC00F0010E546E98EC00F0EAEF00F019
:101EB0004DEF01F0D7EF01F08EEF02F06AEF05F081
:101EC00003C043F002C042F001C041F000C040F046
:101ED000486A496A68EC06F04C0EF66E000EF76E22
:101EE0009DEC06F043C04BF042C04AF041C049F0BF
:101EF00040C048F01BEF08F0486A010E496E68ECDC
:101F000006F0520EF66E000EF76E9DEC06F043C022
:101F10004BF042C04AF041C049F040C048F037D4CD
:101F2000580EF66E000EF76E9DEC06F0C3D7030058
:020000040030CA
:0E00000015C8787C000991000FC00FE00F407A
:00000001FF
